:020000040000FA
:06000000FE300C303A282E
:08000800A000030E8301A1001A
:100010000A08A2008A018A11AA1503140B190310F9
:1000200000308100A30DA40DA50DA90B20282A16D0
:100030002508A8002408A7002308A6001930A90055
:100040008B100B1122088A00210E8300A00E200EB7
:020050000900A5
:040052000034003442
:0C007400203084008001840A80300402E7
:10008000031C3C281F30CE000130CA00CB0080305A
:10009000CD000E30F4003230D70083161F308505B6
:1000A000003086050B3087058312850186018701A4
:1000B000103083168E008312703083168F008312E7
:1000C0000030031799000313003003179A0003133D
:1000D0000C30970000309F00003083169F00831281
:1000E000183003179E000313003003179F000313FB
:1000F000803083168100831211309000043092000A
:100100007F308316920083120030950000308316F2
:100110009400831223309400A63083169800831233
:10012000003083169B00831210309800193083161C
:1001300099008312003083168C00831200308316DE
:100140008D00831200308B000D163A2481018E0140
:100150008F010B118B100B108C018D010D168B175D
:100160001230E00015228A15F9228A1131178921EF
:100170003023FE20661A0521E61A00212A1A0A21D8
:100180008F080319B8288F01E61A0717661A071592
:100190008A1500208A11B11B9821661A0521E61ADA
:1001A00000210F24FC2358220E23E70BE428301EE5
:1001B000DF28B20BDF2830128A15F3228A11401F84
:1001C000E428E30BE4284013661A0521E61A00210F
:1001D0004F18D421661A0521E61A00214F18B828B5
:1001E000AA19F828CC0BB828AA1AFC281930A9009B
:1001F000AA110C30CC00B8288121B828640008006E
:100200006B080E020318071308006B080E02031890
:10021000071108002A12C1302802031D1C292708D3
:10022000BE002608BD0007303E028A1503190D23C3
:100230008A11E0233A247C29280827062602031D78
:10024000080096302802031D32292708BA00390811
:10025000203C031C7C29B91F7C29390884003A08FA
:1002600080007C29B90191302802031D3A29270812
:10027000B9007C29F7302802031D41292708BF0057
:100280007C29A1302802031D48292708F0007C2979
:10029000A2302802031D4F292708C2007C29A7305D
:1002A0002802031D60292A10A71B2A1427087F395A
:1002B000EA002A1CEA012B142A1C2B10AB157C29FE
:1002C000C2302802031D7C292708C40064000D1ECB
:1002D00067298B13440803178D0083168C130C14A5
:1002E00083120C080313C5008B177F304402413082
:1002F0000319C500CE167C29AA16AA110A30CC0013
:1003000008004F144F150B128316051183120515A3
:1003100008004F10CF101930A900AA12AA110A30F4
:10032000CC008316051583128B100B110B160800D9
:10033000E81C080034080319080034083702031DBC
:10034000A72935083802031DA729B1130800AF0AF1
:1003500001302F02031DAF29340893000800073035
:100360002F02031DB6293508930008000D302F0217
:10037000031DC02936080319080036089300080039
:100380000E302F02031D08003408B7003508B800EE
:10039000B401B501B601AF01B113311F08008A15D0
:1003A00003238A11311308004F19E129C9030F30C3
:1003B0004905031D0800C9080319E1290515C90EDF
:1003C000080005114F11CF1889294B184608CB1882
:1003D00047084B1948084D05031DF1294430C90051
:1003E000F4291130C900F4290310CD0C0318F929A0
:1003F00008008030CD000310CB0DCB19002A080077
:100400000130CB001030CE1ACA00410840028030C3
:10041000031DCA000310CA0D03184A144A084E05EA
:100420000319002A1522CF140800C601C701C8010C
:100430004A1C202A7730C6004008C700C100542A51
:10044000CA1C272A6630C6004308C700542A4A1D22
:100450002E2A5530C6007108C700542ACA1D372AF3
:100460004430C6005F08C700FF30DF00542A4A1E30
:100470004A2A3330C6008B13343003178D0083169D
:100480008C130C1483120C08031384008B170008C0
:10049000C700542ACA1E08002130C6004408C700FD
:1004A0004508C800CE12080046084706C8000800E4
:1004B000051C642A401E822A83160313A00383129C
:1004C000031303194012822A401A7C2A831603134D
:1004D000A00A831203138316031324082002831235
:1004E0000313031D822A4016691C822A30168A15BE
:1004F000F3228A110530B200FF3083160313A000E7
:1005000083120313851C8E2AC01DAC2A8316031385
:10051000A103831203130319C011AC2AC019A62A20
:1005200083160313A10A83120313831603132408EB
:10053000210283120313031DAC2AC015E91CAC2A47
:1005400030168A15F3228A110530B200FF30831667
:100550000313A10083120313851DB82A401DD62A58
:1005600083160313A2038312031303194011D62A1F
:100570004019D02A83160313A20A83120313831689
:1005800003132408220283120313031DD62A4015E5
:10059000691DD62A30168A15F3228A110530B20059
:1005A000FF3083160313A200831203138719C010B0
:1005B000871DC0143F1886163F1C8612C2192324BB
:1005C000C219E62A2A1B23242A1F0712E819ED2A3A
:1005D000BF1C8613BF188617F12ABF1C8617BF18C9
:1005E00086133F1F6613401CF82A3F1BF82AE617A4
:1005F000C01C012B681D012B71080319012BF1018F
:10060000DA23C3180A2B2B1C0A2B05307702431060
:10061000031C43146615C21E66110800B11B0800B6
:10062000E008031D08003108420601390319212B97
:100630003013421830178A15F3228A1131104218EC
:10064000311431084206023903190800B110C218EA
:10065000B11430168A15F3228A110530B200080051
:10066000EA0803193A2BAB18442B6A0895002A189C
:100670003C2B080095010800C311431306162B14E8
:10068000AB10421AAB1408002B1D08002B11D51813
:100690008F2BD70B08003230D700D514AB1963234A
:1006A0008B131D3003178D0083168C130C148312CB
:1006B0000C080313DE006A0895002A1C0800AB1022
:1006C000421AAB140800AB112130BF1C013E0317C6
:1006D0008D0083168C130C1483120C080313D8009E
:1006E0008B17203003178D0083168C130C14831284
:1006F0000C080313DC008B1758085C07D9005C0753
:10070000DA005C07DB00303003178D0083168C1392
:100710000C1483120C080313DD008B170800DE088D
:100720000319942BDE03080058087702031CA62B3C
:1007300059087702031CA82B5A087702031CAA2B1E
:100740005B087702031CAC2BD40AAE2BD00AAE2B6D
:10075000D10AAE2BD20AAE2BD30AAE2B50085104CD
:10076000520453045404103903190800D601501AD6
:10077000D614511A5615521AD615531A5616541A1B
:10078000D616D001D101D201D301D401D510323017
:10079000D7006A08ED005D075619ED005D07D61910
:1007A000ED005D07561AED005D07D61AED006D08E5
:1007B000950008000030BE007108BD00E02308006D
:1007C0000D123E08831203178D00831203133D0898
:1007D000831203178C00831603178C130C158B13CD
:1007E0008B1BEF2B55308D00AA308D008C148B178E
:1007F0000C11831203130800F40B0C2C0E30F400C0
:100800009F147503F6009F18032C2A151E08F50087
:100810005F0275080318DF008D309F0008009F14E9
:100820009F18102C2B158B1383161E0883128B1701
:10083000F7001E08C310031DC314FF30C318F700D0
:1008400011309F000800AD132D13AD0B0800AC0A4A
:1008500003302C02031C080007121E302E1C0A3025
:100860002C02031C0800AE0A0130E81AAE0007167D
:10087000AC01080064000D1E3B2C8B1300300317E5
:100880008D0083168C130C1483120C080313F100D3
:100890008B13313003178D0083168C130C148312C5
:1008A0000C0803138B17F2003030F21BF200F20336
:1008B0008B138B1B582C083003178D0083168C1359
:1008C0000C1483120C080313E8008B178B138B1B7B
:1008D000662C093003178D0083168C130C148312B9
:1008E0000C080313E9008B171C3003178D008316C7
:1008F0008C130C1483120C08031383160313A40027
:10090000831203138B1708000708403A870008007A
:100910000708043A870008000708103A8700080013
:100920000608103A860008000608203A86000800EB
:080930000608803A8600080069
:10100000143060020318E00108308A00600882078B
:101010001C283828D728E528F4280D2937294B29FA
:101020007929B329EF291C2A312A3F2A4E2A672A17
:10103000812A962AA12AA82A071707112A1C061214
:10104000FA01FB01EB01E6134010C012C313661B4B
:1010500008003F1F0800421F66173A23F3080319D0
:101060000800421BE810421BE6170130E0000800B0
:10107000AB104014661DB017F3222A17C311431397
:101080008B13053003178D0083168C130C148312F9
:101090000C080313EC008B178B13033003178D0020
:1010A00083168C130C1483120C080313F8008B178F
:1010B0008B13043003178D0083168C130C148312CA
:1010C0000C080313F9008B178B130C3003178D00DA
:1010D00083168C130C1483120C080313FC008B175B
:1010E0008B130D3003178D0083168C130C14831291
:1010F0000C080313FE008B178B130F3003178D00A2
:1011000083168C130C1483120C080313FD008B1729
:101110008B130E3003178D0083168C130C1483125F
:101120000C080313FF008B178B131B3003178D0064
:1011300083168C130C1483120C080313E4008B1712
:101140008B13133003178D0083168C130C1483122A
:101150000C080313E5008B170130BF1C013E8B13F5
:1011600003178D0083168C130C1483120C080313C1
:10117000EF008B171130BF1C013E8B1303178D003E
:1011800083168C130C1483120C080313EE008B17B8
:10119000421BEC010130421BE5006C08E100FF300E
:1011A000EB000230E000EC080319DE280800E61628
:1011B000E10B08006C08E100EB0B0800E612650883
:1011C000E100E2010330E000080007130711E20B21
:1011D0000800E10B08006C08E100EB010430E000BE
:1011E000EC080319FC2808006616E10B08006C08DF
:1011F000E100EB0F0800EB0366128B1314300317AA
:101200008D0083168C130C1483120C080313E10059
:101210008B17E2010530E000080007130715E81CF2
:101220001F2966191F29E10803191F29E81F301615
:10123000E81B3017F322E20B0800E10B0800E81F5F
:101240003012E81B3013F3228B13163003178D0076
:1012500083168C130C1483120C080313E1008B17F4
:10126000E2010130421BE1000630E0000800E20B21
:101270000800E10B08008B13183003178D0083164C
:101280008C130C1483120C080313E1008B17E2017A
:101290000730E0000800C0160616AB156E08EA001D
:1012A000AB14681CAB10E614E0222B14E20B080010
:1012B000E10B08000130E61BF300AB1001307302B4
:1012C000031D69296E08EA00AB14681CAB10E61018
:1012D000CD228B13193003178D0083168C130C1439
:1012E00083120C080313E1008B17E2010830E000C1
:1012F0000800B02278087502031883297F08FB02D2
:10130000031C882908007F08FB070318A22908008E
:10131000FB010130E61BF300AB1001307302031D2B
:1013200098296E08EA00AB14681CAB10E610CD22B9
:10133000E20B0800E10B0800C315F3012A1311307A
:10134000E0000800FB018B131A3003178D00831691
:101350008C130C1483120C080313E1008B17E201A9
:101360000930E0000800B02279087502031CBD298D
:101370007F08FB02031CC22908007F08FB07031833
:10138000CC290800FB01E20B0800E10B0800431721
:10139000F3011130E0000800BF1C5923BF185F2380
:1013A000F31BDF29F30BDF296E08EA00AB14681C7E
:1013B000AB10E610CD220A30E000FA0108008B13D2
:1013C000193003178D0083168C130C1483120C082C
:1013D0000313E1008B17E2010830E00008002A1D2A
:1013E00008002A1175087602031CFB297C08FA0202
:1013F000031C022A08007E08BF1C7D08FA07031898
:10140000042A0800FA010800FA018712EA012B10E9
:10141000AB10C7228B131730421B333003178D00DC
:1014200083168C130C1483120C080313E1008B1722
:10143000E2010B30E00008008A11DA238A15C0129D
:101440000612E20B0800B013F322E10B0800EC08CF
:101450000319382A6C08E100FF30EB000C30E00083
:1014600008006616E10B08006C08E100EB0B0800B1
:1014700066126508E100E2010D30E0000800071384
:101480000711E20B0800E10B08006C08E100EB011A
:101490000E30E000EC080319562A0800E616E10BAE
:1014A00008006C08E100EB0F0800EB03E6128B1359
:1014B000153003178D0083168C130C1483120C083F
:1014C0000313E1008B17E2010F30E000080007175B
:1014D0000711E81C792A6619792AE1080319792A83
:1014E000681F3016681B3017F322E20B0800E10B6F
:1014F0000800681F3012681B3013F3221030E00020
:1015000008002A13C7228B13323003178D0083166D
:101510008C130C1483120C080313E3008B1771084F
:101520007002031940170030E00008002A13C72298
:10153000B0138712EA012B10AB1006120030E00046
:101540000800C3171430E100E2011330E000080086
:10155000C317E20B0800E10B08000030E0000800B0
:10156000E61C0800E40B08008B131B3003178D00EA
:1015700083168C130C1483120C080313E4008B17CE
:10158000EA0A6F086A02031D0800E610080024300A
:10159000B4000030B500B11708002430B4008B133C
:1015A0001E3003178D0083168C130C1483120C0845
:1015B0000313B6008B178A1529238A15B117080063
:1015C0002430B4008B131F3003178D0083168C1347
:1015D0000C1483120C080313B6008B178A152923E9
:1015E0008A15B11708000630B4003008B500B117ED
:1015F00008001430AF00FE30B400D930B500FF3021
:10160000B600B11708001430AF00FE30B400E5306A
:10161000B500FF30B600B1170800B701FE30B400C6
:10162000A130B5008A1517238A15B1170800B60135
:101630003D18B617BD1836173D19B616BD19361622
:101640003D1AB615BD1A36153D1BB614BD1B361412
:101650000800B5013618B517B61835173619B5167E
:10166000B6193516361AB515B61A3515361BB51412
:10167000B6010800701B562B700871020319542B19
:1016800003184C2B03194C2B71087002BF187202FF
:10169000BF18013EF300080070087102BF1C7202FF
:1016A000BF1C013EF3000800F3010800FA30F3000C
:1016B0000800F10A720A71020318F1000800F10330
:0816C000720AF11BF10708009A
:084000000B000000000041006C
:02400E00CC03E1
:1042000000007E007E00AA0096000A001800FF0051
:1042100087000000FF00FF0041002E0014002E0068
:1042200000003200320002001400150016003700B2
:104230000600190080005A00FF000A00010060001B
:10424000050040004000FF00FF00FF00FF00FF00EE
:10425000FF00FF00FF00FF00FF00FF00FF00FF0066
:104260000A00FF000F0022007700FF00FF00FF00A0
:10427000FF00FF00FF00FF00FF00FF00FF00FF0046
:10428000FF00FF00FF00FF00FF00FF00FF00FF0036
:10429000FF00FF00FF00FF00FF00FF00FF00FF0026
:1042A000FF00FF00FF00FF00FF00FF00FF00FF0016
:1042B000FF00FF00FF00FF00FF00FF00FF00FF0006
:1042C000FF00FF00FF00FF00FF00FF00FF00FF00F6
:1042D000FF00FF00FF00FF00FF00FF00FF00FF00E6
:1042E000FF00FF00FF00FF00FF00FF00FF00FF00D6
:1042F000FF00FF00FF00FF00FF00FF00000039008B
:10430000FF00FF00FF00FF00FF00FF00FF00FF00B5
:10431000FF00FF00FF00FF00FF00FF00FF00FF00A5
:10432000FF00FF00FF00FF00FF00FF00FF00FF0095
:10433000FF00FF00FF00FF00FF00FF00FF00FF0085
:10434000FF00FF00FF00FF00FF00FF00FF00FF0075
:10435000FF00FF00FF00FF00FF00FF00FF00FF0065
:10436000FF00FF00FF00FF00FF00FF00FF00FF0055
:10437000FF00FF00FF00FF00FF00FF00FF00FF0045
:10438000FF00FF00FF00FF00FF00FF00FF00FF0035
:10439000FF00FF00FF00FF00FF00FF00FF00FF0025
:1043A000FF00FF00FF00FF00FF00FF00FF00FF0015
:1043B000FF00FF00FF00FF00FF00FF00FF00FF0005
:1043C000FF00FF00FF00FF00FF00FF00FF00FF00F5
:1043D000FF00FF00FF00FF00FF00FF00FF00FF00E5
:1043E000FF00FF00FF00FF00FF00FF00FF00FF00D5
:1043F000FF00FF00FF00FF00FF00FF00FF00FF00C5
:00000001FF
